:20000000facd28c014c000c0dfb69f938f93ff93ef93e0916800f0916900cf01892b09f060
:200020000995ef91ff918f919f91dfbe1895bfb69f938f93ff93ef93e0916400f0916500e0
:20004000cf01892b09f00995ef91ff918f919f91bfbe1895cfb69f938f93ff93ef93e0919d
:200060006600f0916700cf01892b09f00995ef91ff918f919f91cfbe1895f89496958795aa
:2000800090936500809364008991999178940895f894969587959093670080936600899184
:2000a000999178940895f89496958795909369008093680089919991789408959a938a935c
:2000c00088279927dacf9a938a9388279927e0cf9a938a9388279927e6cff894969587955f
:2000e0009093610080936000899199917894089596958795fc018991999109949a938a93ad
:200100000895688179819a938a93cb01089569917991089500d08991999108956991799156
:20012000f2cf2f903f909f938f933f922f92f3cf2f903f906f917f913f922f92e4cf00d015
:20014000f0dfecdff5dfeacf80959095089581952224290a922d0895880f991f08959595a0
:20016000879508959695fccff2df69917991860f971f089569917991862397230895699115
:200180007991862b972b0895699179918627972708959a938a93fb0101c0fc018191919101
:2001a00008959a938a93fb0101c0fc01819199270895fb0103c0fc018991999181939193f7
:2001c000aacffb0103c0fc01899199918193a3cf892b8150880b982f0895990ffbcf699138
:2001e0007991681b790b08959a938a93cb01f7dff1cf9a938a93cb01f2df14f40894eacf61
:200200008894e8cf9a938a93cb01e9df11f40894e1cf8894dfcffc01859195910895fc013f
:200220008591992708959a938a93f89480915d0090915e0078949a938a93f701d583c4839b
:20024000e280f380f70180818823d1f3c481d58189919991f89480935d0090935e007894f9
:200260008991999108958dea9eed08956ae672e09a938a93cb016be670e09bcf66e272e0a1
:200280009a938a93cb016be670e093cfe0916b00f0916c00f695e7950994e0916f00f09177
:2002a0007000df01fe97880f991f06969f01e81bf90bf0937000e0936f0000270083818344
:2002c000b383a283cf01e0916d00f0916e0093838283089596958795a991b991fd0101e0c4
:2002e000008301811127e00ff11f34971496ed93fd93df01ff96ed93fd9391838283899185
:2003000099910895fe01fc977f0101e000830ce30183f382e282f0927000e0926f00f092ff
:200320006e00e0926d000895b1df0895a89501b5086101bd00e001bd0895c0916200d0913d
:200340006300ee97002492df8edff0dfdbdf68e273e09a938a93cb01c0deb0deb9ce595219
:200360002050532f32207620302e3920323031390196089501970895002704bd00e408bf24
:20038000089567e070e09a938a93cb0165e470e018dff2cf9a938a93882708b706ff03c042
:2003a0008fef007408bf982f089560e070e09a938a93cb01a3de61e970e003df62e970e0e2
:2003c00000cf8f71089562e970e0ebde61e970e0e8de1bcf93dee9dea1de93dec9df9edeb7
:2003e000f2ce61e970e09a938a93cb01f3dfe9df61e770e0bcded9ce979a08959798089580
:20040000969a0895969808959598880f10f4c09a01c0c098959a0895f5df68e070e09a93a4
:200420008a93cb01bf93af93dc0189919991ecdf1197e9f7af91bf916edee2cf61e370e0aa
:20044000b0de60ee70e09dde61e370e0baded4cf88980895889a089589980895899a08952c
:200460008c9808958c9a0895a5980895a59a0895a4980895a49a0895a2980895a29a0895de
:20048000a1980895a19a0895a0980895a09a0895a3980895a39a08950895c19a0895c19862
:2004a0000895c79a0895c7980895c39a0895c3980895c59a0895c5980895c69a0895c69862
:2004c0000895c29a0895c2980895c49a0895c498089563e970e065de9fcfa3e9b0e00c9195
:2004e000012b0c930895a3e9b0e00c9101230c93089511e0f2cf1eeff6cf14e0eecf1bef3c
:20050000f2cf18e0eacf17efeecf10e1e6cf1feeeacf10e2e2cf1fede6cf10e4decf1feb2b
:20052000e2cf12e0dacf1defdecf10e8d6dfd1cf1fe7d9dfcecfb0cfb0cfb3cfb6cfb9cf81
:20054000bccfbfcfc2cfa8cfaacfadcfb0cfb3cfb6cfb9cfbccf7ecf81cfe7cf83cf86cff2
:2005600089cf8ccf8fcf92cf95cf0895089508950895089508956ccf6fcfdacf71cf74cf52
:2005800077cf7acf7dcf80cf83cf089508950895089508950895e6dde5dde4dd6ee170e04c
:2005a000ebcdacdd60e870e0e7dddcdddbddb6dd6fe070e0e1ddd0dde2cd60e870e0e1cd9b
:2005c0009dddefdf66e575e0d2dd92dde4df66e375e0cddd8dcd8a418a723110308a8a8ada
:2005e000002062118a8a8a8a8a8a8a18148a8a8a29381678248a8a3609465644348a8a8ac0
:2006000068664828548a8a6726077619648a8a8a57275874058a8a4537177704158a8a6510
:2006200075473508558a8a8a8a8a398a8a8a8a8a21598a498a8a8a8a8a8a8a8a038a8a1407
:200640008a44748a8a8a046524546405308a8a8a34558a158a8a8a8a8a408a8a8a418a72ad
:200660003110308a8a8a002062118a8a8a8a8a8a8a27148a8a8a18196636248a8a3869781b
:200680005844348a8a8a57165637548a8a4817280867648a8a8a09777674058a8a26473969
:2006a0005904158a8a0665466829558a8a8a498a078a8a8a8a8a21798a498a8a8a8a8a8a4a
:2006c0008a8a038a8a148a44748a8a8a046524546405308a8a8a34558a158a8a8a8a8a40c9
:2006e0008a8a8a8a8a8a8a8a8a8a8a8a8a8a8a8a8a8a8a8a8a8a8a8a8a8a8a8a8a8a8a8aba
:200700008a618a8a8a8a8a8a8a718a8a8a8a8a8a8a328a8a8a8a8a8a8a8a8a8a8a8a8a8a33
:200720008a8a8a8a8a8a8a8a8a8a8a8a758a8a8a8a8a8a8a8a8a8a8a8a8a8a8a218a8a8af7
:200740008a8a8a8a8a8a8a8a8a8a8a8a8a018a8a8a8a3262338a13238a8a8a8a8a8a8a8a97
:200760008a8a8a8a8a8a8a8a68e970e012dd66e970e01fcd62ee76e09a938a93cb0166e903
:2007800070e017cd66ed75e09a938a93cb0108956ce576e09a938a93cb01089568e970e0cf
:2007a00008dde2cffc0189919991e80ff91f992784910895a3dc66e870e01bddc5dc982b68
:2007c0008991999131f0a7dc60e070e09a938a93cb0166e970e0dddce5cfecdff1ceeadf2c
:2007e000ecdeeece6de970e0d4dc64e970e0e1dcbbcf6fe970e0cddc64e970e0dadcb4cf12
:2008000061ea70e0c6dc64e970e0d3dcb3cf63ea70e0bfdc64e970e0ccdcaccf65ea70e036
:20082000b8dc64e970e0c5dc60e070e09a938a93cb016ce970e0c5cc9fdd28ddabdd982b3e
:2008400089919991d1f30895bbdef6cf51dc41def3cf60e070e09a938a93cb015fdcb3cc27
:20086000a4dcb6cc6fef7fef9a938a93cb0156dcaacc9bdcaddc68cc60e070e09a938a93de
:20088000cb0163e970e09ddc67ea70e09a938a93cb01dfdf68ea70e09a938a93cb01d9df92
:2008a00069ea70e09a938a93cb01d3df6aea70e09a938a93cb01cddf6bea70e09a938a9378
:2008c000cb01d0df6cea70e09a938a93cb01c1cf6fef7fef9a938a93cb0120dc0fdc61e146
:2008e00070e090dc982b8991999171f014dc05de68ea70e09a938a93cb01b4df6aef74e009
:200900009a938a93cb01a2cff9db62e170e07adc982b8991999171f0fedbf7dd6aea70e0da
:200920009a938a93cb019edf6ae075e09a938a93cb018ccfe3db64e170e064dc982b8991a4
:20094000999171f0e8dbdddd67ea70e09a938a93cb0188df62e075e09a938a93cb0176cf7f
:20096000cddb69e270e04edc982b8991999141f0d2dbd7dd62e275e09a938a93cb0166cf8d
:20098000bddb68e570e03edc982b8991999139f1c2db6bea70e09a938a93cb016adf982b73
:2009a0008991999171f0b9dd6bea70e09a938a93cb014fdf6ae175e09a938a93cb0146df38
:2009c0000dc0a7dd6bea70e09a938a93cb014adf62e175e09a938a93cb0138df08958edb17
:2009e00069e570e00fdc982b8991999171f093db8cdd6aea70e09a938a93cb0133df6ae019
:200a000075e09a938a93cb0121cf84db60e070e09a938a93cb0108956fef7fef9a938a93c3
:200a2000cb017cdb6bdb6ee170e0ecdb6aea70e09a938a93cb011ddf9ddb982b89919991b2
:200a400099f069db6ee075e09a938a93cb01fede66e070e09a938a93cb01f6de6cea70e00e
:200a60009a938a93cb01fece49db66e370e0cadb6aea70e09a938a93cb01fbde7bdb982b86
:200a80008991999199f047db6ee075e09a938a93cb01dcde69e670e09a938a93cb01d4de8d
:200aa0006cea70e09a938a93cb01dcce27db6de370e0a8db6aea70e09a938a93cb01d9de3a
:200ac00059db982b8991999169f025db64e670e09a938a93cb01b8de6cea70e09a938a934c
:200ae000cb01c0ce0bdb61e470e08cdb6aea70e09a938a93cb01bdde3ddb982b8991999146
:200b000069f009db65e470e09a938a93cb019cde6cea70e09a938a93cb01a4ceefda6ce428
:200b200070e070db6aea70e09a938a93cb01a1de21db982b8991999199f0edda6ee075e0eb
:200b40009a938a93cb0182de65e270e09a938a93cb017ade6cea70e09a938a93cb0182ce0e
:200b6000cdda62e570e04edb982b8991999121f1d2da6aea70e09a938a93cb0171de982b7d
:200b80008991999169f0c7da6ae075e09a938a93cb015cde64e770e09a938a93cb0154ce55
:200ba00064e270e09a938a93cb014ede6cea70e09a938a93cb0156cea1da64e570e022db6c
:200bc0006aea70e09a938a93cb0153ded3da982b8991999169f09fda64e070e09a938a93c6
:200be000cb0132de6cea70e09a938a93cb013ace85da6be570e006db6aea70e09a938a9387
:200c0000cb0137deb7da982b8991999199f083da6ee075e09a938a93cb0118de69e770e026
:200c20009a938a93cb0110de6cea70e09a938a93cb0118ce6fda60e070e09a938a93cb011f
:200c400008956fef7fef9a938a93cb0167da56da6ee170e0d7da6aea70e09a938a93cb019a
:200c600008de88da982b8991999169f054da64e270e09a938a93cb01e7dd6cea70e09a935b
:200c80008a93cb01efcd3ada65e270e0bbda6aea70e09a938a93cb01ecdd6cda982b8991c9
:200ca000999199f038da6ee075e09a938a93cb01cddd65e370e09a938a93cb01c5dd6cea66
:200cc00070e09a938a93cb01cdcd18da66e370e099da6aea70e09a938a93cb01cadd4ada91
:200ce000982b8991999199f016da6ee075e09a938a93cb01abdd65e270e09a938a93cb0186
:200d0000a3dd6cea70e09a938a93cb01abcdf6d96de370e077da6aea70e09a938a93cb01a5
:200d2000a8dd28da982b8991999169f0f4d965e770e09a938a93cb0187dd6cea70e09a9316
:200d40008a93cb018fcddad96ae470e05bda6aea70e09a938a93cb018cdd0cda982b8991e2
:200d6000999199f0d8d96ee075e09a938a93cb016ddd65e470e09a938a93cb0165dd6ceac5
:200d800070e09a938a93cb016dcdb8d96de570e039da6aea70e09a938a93cb016addead9a9
:200da000982b8991999199f0b6d96ee075e09a938a93cb014bdd65e770e09a938a93cb0181
:200dc00043dd6cea70e09a938a93cb014bcda2d960e070e09a938a93cb0108956fef7fef95
:200de0009a938a93cb019ad989d96ee370e00ada6aea70e09a938a93cb013bddbbd9982b5a
:200e00008991999169f087d96cea70e09a938a93cb0128dd65e270e09a938a93cb0114cd86
:200e20006dd965e470e0eed96aea70e09a938a93cb011fdd9fd9982b8991999169f06bd93a
:200e40006cea70e09a938a93cb010cdd65e170e09a938a93cb01f8cc51d966e470e0d2d90e
:200e60006aea70e09a938a93cb0103dd83d9982b8991999169f04fd96cea70e09a938a9304
:200e8000cb01f0dc65e070e09a938a93cb01dccc35d965e570e0b6d9982b8991999119f11f
:200ea0003ad96aea70e09a938a93cb01d9dc982b8991999161f06ae075e09a938a93cb01a3
:200ec000c5dc65e570e09a938a93cb01bdcc6cea70e09a938a93cb01c5dc65e370e09a9316
:200ee0008a93cb01b1cc0ad969e770e08bd9982b89919991b9f00fd96aea70e09a938a931f
:200f0000cb01aedc982b8991999131f06ae075e09a938a93cb019adc65e370e09a938a9346
:200f2000cb0192ccebd86ce770e06cd9982b8991999199f0f0d86ae075e09a938a93cb01cf
:200f400085dc6cea70e09a938a93cb018bdc65e270e09a938a93cb0177cc69ea70e09a934d
:200f60008a93cb017ddc982b8991999119f0c6d853dd02c0c3d865de982b8991999109f0b1
:200f8000cac8c8d860e070e09a938a93cb0108956fef7fef9a938a93cb01c0d8afd861e199
:200fa00070e030d9982b8991999171f0b4d8a7da68ea70e09a938a93cb014bdc6eef74e0d3
:200fc0009a938a93cb0142cc99d862e170e01ad9982b8991999171f09ed899da6aea70e001
:200fe0009a938a93cb0135dc6ee075e09a938a93cb012ccc83d864e170e004d9982b89916f
:20100000999171f088d87fda67ea70e09a938a93cb011fdc66e075e09a938a93cb0116cc47
:201020006dd869e270e0eed8982b8991999141f072d879da66e275e09a938a93cb0106ccb0
:201040005dd868e570e0ded8982b89919991d9f062d86bea70e09a938a93cb010adc982b9a
:201060008991999141f057da66e175e09a938a93cb01ecdb07c053da6ee175e09a938a936f
:20108000cb01e4db08953ad869e570e0bbd8982b8991999171f03fd83ada6aea70e09a9381
:2010a0008a93cb01d6db6ee075e09a938a93cb01cdcb30d860e070e09a938a93cb010895fa
:2010c0006aea70e09a938a93cb01d3db982b8991999131f06ae075e09a938a93cb01b6db3a
:2010e00008956fef7fef9a938a93cb0117d806d86ee170e087d86cea70e09a938a93cb01ea
:20110000b8db38d8982b8991999171f004d866e870e09a938a93cb0197dbd2df6cea70e06b
:201120009a938a93cb0195cbe9d766e370e06ad86cea70e09a938a93cb019bdb1bd8982bb6
:201140008991999171f0e7d769ee70e09a938a93cb017adbb5df6cea70e09a938a93cb01ca
:2011600078cbccd76de370e04dd86cea70e09a938a93cb017edbfed7982b8991999169f07a
:20118000cad764ee70e09a938a93cb015ddb6cea70e09a938a93cb015ccbb0d761e470e0bf
:2011a00031d86cea70e09a938a93cb0162dbe2d7982b8991999169f0aed765ec70e09a93c1
:2011c0008a93cb0141db6cea70e09a938a93cb0140cb94d76ce470e015d86cea70e09a9378
:2011e0008a93cb0146dbc6d7982b8991999171f092d765ea70e09a938a93cb0125db60df83
:201200006cea70e09a938a93cb0123cb77d762e570e0f8d7982b8991999119f17cd76ceab6
:2012200070e09a938a93cb011bdb982b8991999161f064ef70e09a938a93cb0105db6ee013
:2012400075e09a938a93cb0101cb6cea70e09a938a93cb01feda64ea70e09a938a93cb010f
:20126000f3ca4cd764e570e0cdd76cea70e09a938a93cb01feda7ed7982b8991999169f008
:201280004ad764e870e09a938a93cb01ddda6cea70e09a938a93cb01dcca30d76be570e0bb
:2012a000b1d76cea70e09a938a93cb01e2da62d7982b8991999199f02ed769ef70e09a938b
:2012c0008a93cb01c1da6ae075e09a938a93cb01bdda6cea70e09a938a93cb01baca1ad70d
:2012e00060e070e09a938a93cb0108956fef7fef9a938a93cb0112d701d76ee170e082d710
:201300006cea70e09a938a93cb01b3da33d7982b8991999171f0ffd664ea70e09a938a9355
:20132000cb0192dacdde6cea70e09a938a93cb0190cae4d665e270e065d76cea70e09a9354
:201340008a93cb0196da16d7982b8991999171f0e2d665eb70e09a938a93cb0175dab0de94
:201360006cea70e09a938a93cb0173cac7d666e370e048d76cea70e09a938a93cb0179da10
:20138000f9d6982b8991999171f0c5d665ea70e09a938a93cb0158da93de6cea70e09a9350
:2013a0008a93cb0156caaad66de370e02bd76cea70e09a938a93cb015cdadcd6982b899181
:2013c000999169f0a8d665ef70e09a938a93cb013bda6cea70e09a938a93cb013aca8ed619
:2013e0006ae470e00fd76cea70e09a938a93cb0140dac0d6982b8991999171f08cd665ece2
:2014000070e09a938a93cb011fda5ade6cea70e09a938a93cb011dca71d66de570e0f2d6e1
:201420006cea70e09a938a93cb0123daa3d6982b8991999171f06fd665ef70e09a938a93df
:20144000cb0102da3dde6cea70e09a938a93cb0100ca60d660e070e09a938a93cb010895ca
:201460006fef7fef9a938a93cb0158d647d66ee370e0c8d66cea70e09a938a93cb01f9d972
:2014800079d6982b8991999169f045d66cea70e09a938a93cb01ddd965ea70e09a938a9327
:2014a000cb01d2c92bd665e470e0acd66cea70e09a938a93cb01ddd95dd6982b89919991fd
:2014c00069f029d66cea70e09a938a93cb01c1d965e970e09a938a93cb01b6c90fd666e4fc
:2014e00070e090d66cea70e09a938a93cb01c1d941d6982b8991999169f00dd66cea70e0e0
:201500009a938a93cb01a5d965e870e09a938a93cb019ac9f3d565e570e074d6982b899198
:20152000999119f1f8d56cea70e09a938a93cb0197d9982b8991999161f065ed70e09a9357
:201540008a93cb0181d96ee075e09a938a93cb017dc96cea70e09a938a93cb017ad965ebea
:2015600070e09a938a93cb016fc9c8d569e770e049d6982b89919991c1f0cdd565eb70e077
:201580009a938a93cb0160d96aea70e09a938a93cb0166d9982b8991999131f06ee075e038
:2015a0009a938a93cb0152d90895a8d56ce770e029d6982b8991999199f0add56cea70e076
:2015c0009a938a93cb0145d965ea70e09a938a93cb013ad96ee075e09a938a93cb0136c957
:2015e00069ea70e09a938a93cb013ad9982b8991999119f083d575dd02c080d577de982b36
:201600008991999109f087c585d560e070e09a938a93cb0108956fef7fef9a938a93cb01c2
:201620007dd56cd561e170e0edd5982b8991999179f071d562d768ea70e09a938a93cb011c
:2016400011d96aef74e09a938a93cb01ffd8cac855d564e170e0d6d5982b8991999179f09a
:201660005ad54fd767ea70e09a938a93cb01fad862e075e09a938a93cb01e8d8b3c83ed591
:201680006fe170e0bfd5982b8991999181f043d569ea70e09a938a93cb01e4d879d87ed86a
:2016a00061e670e09a938a93cb01ced89bc826d567e270e0a7d5982b8991999181f02bd5ec
:2016c00069ea70e09a938a93cb01c3d85bd866d861e770e09a938a93cb01b6d883c81ad5cf
:2016e00060e070e09a938a93cb0108956fef7fef9a938a93cb0112d501d56ae770e082d510
:20170000982b8991999171f006d56aef74e09a938a93cb019bd863e370e09a938a93cb01a4
:2017200093d860c8ebd46de770e06cd5982b8991999171f0f0d46aef74e09a938a93cb0183
:2017400085d863e270e09a938a93cb017dd84ac8e1d460e070e09a938a93cb0108956fefc4
:201760007fef9a938a93cb01d9d4c8d461e170e049d5982b8991999179f0cdd4c0d668eaf3
:2017800070e09a938a93cb0164d86eef74e09a938a93cb015bd826c8b1d464e170e032d59e
:2017a000982b8991999179f0b6d4add667ea70e09a938a93cb014dd866e075e09a938a93eb
:2017c000cb0144d80fc8a6d460e070e09a938a93cb0108956fef7fef9a938a93cb019ed439
:2017e0008dd469e670e00ed5982b89919991d1f092d462e370e09a938a93cb0125d862ebe3
:2018000070e09a938a93cb011fd863e170e09a938a93cb0119d863e970e09a938a93cb011e
:2018200013d8e0c76bd46ce670e0ecd4982b89919991d1f070d462e370e09a938a93cb01be
:2018400003d862eb70e09a938a93cb01fdd761e070e09a938a93cb01f7d761e870e09a93eb
:201860008a93cb01f1d7bec749d46ae770e0cad4982b8991999171f04ed463eb70e09a9381
:201880008a93cb01e1d76eef74e09a938a93cb01ddd7a8c733d46de770e0b4d4982b8991ad
:2018a000999171f038d463ea70e09a938a93cb01cbd76eef74e09a938a93cb01c7d792c77e
:2018c00029d460e070e09a938a93cb01089516d460ef70e097d4982b8991999111f01bd4dd
:2018e00088c70cd460ee70e08dd4982b8991999111f011d48cc702d461ee70e083d4982beb
:201900008991999111f007d489c7f8d3e1d7982b8991999109f0ffc3f1d360da982b899137
:20192000999109f0f8c359c7e9d360ef70e06ad4982b8991999111f0eed354c7dfd360ee2c
:2019400070e060d4982b8991999111f0e4d34ac7d5d31edb982b8991999111f0dcd342c7d2
:20196000cdd37edd982b8991999111f0d4d33ac736d738c7c3d360ef70e044d4982b899186
:20198000999111f0c8d33cc7b9d360ee70e03ad4982b8991999111f0bed324c7afd33bde27
:2019a000982b8991999111f0b6d31cc7a7d39ede982b8991999111f0aed314c70ed712c79b
:2019c0009dd360ef70e01ed4982b8991999111f0a2d308c793d360ee70e014d4982b8991f1
:2019e000999111f098d3fec689d3b9de982b8991999111f090d3f6c681d3ecde982b899178
:201a0000999111f088d3eec6ead6ecc61477e1f014f077006ce07ae19a938a93cb016ce931
:201a200070e0bfd3a2d3fc0199278491eed38cd3982b8991999109f0d5c66ce970e0b1d399
:201a400097d45cd367e070e0d4d3982b8991999119f06ce970e0b5c35ed362ef74e09a937e
:201a60008a93cb01f3d666ef74e09a938a93cb01edd6b8c687d692d66eec78e19a938a93f2
:201a8000cb016de970e095d368e279e19a938a93cb016fe970e08dd360ec79e19a938a93ba
:201aa000cb0161ea70e085d364e779e19a938a93cb0163ea70e07dd364e17ae19a938a93d5
:201ac000cb0165ea70e075d38dc664e970e061d30fc3dcd378d47cd3982b8991999111f00b
:201ae00080d4f3dff6cf08956be070e09a938a93cb016dea70e065c304e003bf08950f92fa
:201b0000bf93af930f9300248fef08b700ff03c0882701e008bfadeab0e0882311f40be053
:201b20000c9309ef02bf0c91033048f00b3038f4839b88948091ae0087958093ae000c916b
:201b40000a9579f480919200982f9395909392008f71a1e7b0e0a80fb01d8091ae008c93b8
:201b60000be00093ad000f91af91bf910f9008956be570e016d360e470e09a938a93cb019b
:201b8000e3d2f8d26be570e01cc36be570e009d360e470e0f6d26be570e013c30091550013
:201ba0000c7f0260009355008a9892988b98939808950fef07bb42d48cd420c45dd6f9dff4
:201bc000eddff3d399dfddd38fdf6eef7ae19a938a93cb0168c24edfcbdff0dfd6cf64e155
:201be00070e09a938a93cb0158d362ed7ae19a938a93cb016fc3a1d341d3eddff0df46d326
:041c0000fecf089576
:201f000062c081c0ffffffff7dc0ffffffffffffffff77c0ffffffffffffffffffffffff02
:201f2000ffffffffffffff93ef93e0916000f09161000995ef91ff915f9bf5cf0cb108951a
:201f4000fbdfe02ff9dff02f0895fadf04915d9bfecf0cb90895f4dfefdf00830895f0dfdf
:201f60000081f5cfeddf099417b710fdfdcf1fb7f894e199fecf27bfe8951fbf0895e0dfc6
:201f8000df01dedf23e0f0df21e1eedf60e40d901d9021e0e9df32966250c9f7e054f0400e
:201fa00025e0e2df21e1e0df67b766fdfbcf0895003089f2013099f2023009f3033029f2cf
:201fc000043081f2089561e06bbf62e06bbf6eef6dbf6093620063e06ebf609363006ce0f6
:161fe00069b960e060bd0aea1fe01093610000936000789405c0b1
